:030000000219FDE5
:03000B000200A848
:03002B0002015B74
:03005B000202ECB2
:030073000202D9AD
:1000800002030406080C10182030406080040608A3
:100090000C10182030406080A0C00003070F1F051F
:1000A000050D050305030302C2AFC0D0C0E0206206
:1000B00014E5256009E473E525F4F58AD262D0E001
:1000C000D0D0D2AF3285268AC262E526F4603030C5
:1000D000682620720DD0E0D0D0C290C291C292D2D8
:1000E000AF32C290C291C292206F0D20650A740196
:1000F000D5E0FDE57BF45290D0E0D0D0D2AF3275A0
:100100008A00C28DD26201F801B73068052065020D
:10011000D29001B7306805206502D29101B73068EE
:1001200005206502D29201B7D29330680A20650794
:100130007405D5E0FDD29001B7D29430680A2065ED
:10014000077405D5E0FDD29101B7D29530680A2039
:1001500065077405D5E0FDD29201B7C2AFC2AD53B9
:10016000E6EFC0D0C0E0D2D3D2AFC2CEE52A60075E
:1001700020744F152A21C27800790020742EE58062
:10018000307E01F430E70278FF53DACF207E03435C
:10019000DA20307E0343DA10C2D8C271E580307EA7
:1001A00001F430E70279FFC3E89970CB3061037541
:1001B0002A18207403752A18885CD270E8600375C9
:1001C0005F0020740DE52B6004152B21D243DA016A
:1001D000C2D82070024145A85C206102C270207420
:1001E00031C3E894F0400374F0F8E8C4540F28F8E1
:1001F0007984B703024112C313C313872120080275
:10020000C313200A06C3C898F8411228F850037493
:10021000FFF8C3E895655003E565F88822E52D549D
:10022000066022206B1FE536C333C333F8E564C391
:1002300013C313F9C3952240028922E82522F5222F
:1002400050037522FF852224A824C3E5249561402C
:1002500002A8618825E56670024189C3E8AA669A0A
:100260005003E8FAE4F9EAC333FBE568F45B29409C
:100270000D2567F8E56760021567400B41890AC3E1
:10028000E5679A5002056778FF8826C26FC3E526A6
:1002900094F84002D26F20CF0AD0E0D0D043E610CD
:1002A000D2AD32C2CF053A7801E52A60053074023A
:1002B000152AC3E55C94014005755F0041CF756068
:1002C00000756900E55F2401F55F5003755FFFD09D
:1002D000E0D0D043E610D2AD32C2AF53E67F759284
:1002E000FA7593FFC260759104D2AF32C2AF53E684
:1002F000EFC2ADC0D0C0E0C0F0D2D3D2AFA8FBA94E
:10030000FCC2D8307102615353DACF207E0343DA46
:1003100010307E0343DA20D271E580307E01F42074
:10032000E702612A88278928A18053DACF207E033B
:1003300043DA20307E0343DA10C2D8C2713074022F
:10034000A16C7800E580307E01F430E702A16C8872
:100350005CA15453DACF207E0343DA20307E03437E
:10036000DA10C271206102812C53DACF207E034360
:10037000DA10307E0343DA20C2D8D2718857895808
:10038000C3E89555F8E99556F97B007E087A00C3D5
:10039000E8948CE994005005755B00811E882178F3
:1003A000A2E6A8216055C3E894C8E994005008E487
:1003B000D2E4FB7A0A61F9C3E89468E99401500831
:1003C000E4D2E3FB7A0F61F9C3E894D0E9940250D8
:1003D00008E4D2E2FB7A1E61F9C3E894A0E994052F
:1003E0005008E4D2E1FB7A3C61F9C3E89498E994BF
:1003F000085008E4D2E0FB7A787E00C3E89559FC07
:10040000E9955AFD30E70AECF42401FCEDF43400E0
:10041000FD755B00C3EC9AED9E5003755B01885936
:10042000895A8557558558567802A154C3E89527AF
:10043000F8E99528F9307C02A138307B02A13830E8
:100440007A02A131207502814FE9FDE8FC816EE955
:10045000C313F9E813F8307902A131E9C313F9E8BD
:1004600013F8307802A131E9C313FDE813FC2061D1
:0F0470002CC3EC941CED940240028185ED701EAC
:10047F00C3EC94C850180529E52970021529C3E566
:10048F0029940A5002A16C755C00D270A16CE52909
:10049F00600215297888E6F97400207F087896B9EC
:1004AF000302789EE624FAFEE43400FFC3EC9EFCC0
:1004BF00ED9FFD9208B90310A2085007207609D2CC
:1004CF007681D7307602C276A2085016B9030DECAA
:1004DF00F42401FCEDF43400FD0204F178007900FE
:1004EF00A138B90315EC33FCED33FDC3EC940AFCD2
:1004FF00ED9400FD50047C007D00C3EC94FFED945F
:10050F0000400678FF7900A138EC8572F0A4C5F0A1
:10051F00A2F733F87900400302055478FF790002FF
:10052F000554E9C313F9E813F8307C0EE96002783B
:10053F00FFC3E81338F8E43400F9C3E894FFE994F3
:10054F0000400278FF885CD270206102A16C741F9A
:10055F00F4552F4BF52FC274EB7002D274752A1815
:10056F00307403752A0A306102A18020740353DAB4
:10057F00FE207403752B06D0F0D0E0D0D0D2AD435F
:10058F00E6103279010205B079030205B0790A024B
:10059F0005B0791E0205B079640205B079C802056D
:1005AF00B07817E4D5E0FDD8FAD9F6227A147B7823
:1005BF000205D77A107B8C0205D77A0D7BB4020522
:1005CF00D77A0B7BC80205D7E573D5E001227902F4
:1005DF00E4D294D5E0FDD291D5E0FDC291D5E0FDF6
:1005EF00C294D5E0FDE920E002D29030E002D29231
:1005FF00E573D5E0FDE920E002C29030E002C2923F
:10060F007496D5E0FDD9C9EAF8D5E0FDD8FBDBB883
:10061F00D29422C37C007D0075F00005F0EA33FA16
:10062F00EB33FB50F6EB13FBEA13FAC3E9FFE8FEDB
:10063F00E89AF8E99BF95004EFF9EEF8B3EC33FCC4
:10064F00ED33FDD5F0DFEDF9ECF822E889F08A20E3
:10065F00D2D4F8A9F07B0030F70B7BFFF42401F81C
:10066F00E9F43400F9E88520F0A4ADF0F8E985202D
:10067F00F0A4AFF0FEED2EF974003FFA7C04C3EA4C
:10068F0013FAE913F9E813F8DCF48BF030F70AE802
:10069F00F42401F8E9F43400F9E889F0C2D4F8A998
:1006AF00F02222C3E54113F9E54013F8C3E544985E
:1006BF00F8E54599F9500CC3E89480E994FF40168A
:1006CF000206E9C3E8947FE9940050030206E97833
:1006DF007F79000206E9788079FF8849894A22E507
:1006EF00492546F8E54A3547F9854A20E4300701A0
:1006FF00F43548FA30E709C3EA94F04015020727AA
:10070F00C3EA940F500302072778FF79FF7A0F028D
:10071F000727780079007AF0C3E5249561500AC362
:10072F0074019524500B020745E54A20E70E020796
:10073F0045E54A30E706884689478A482278A5E684
:10074F00FAC3E54933F8E54A33F9D15AE930E70BF3
:10075F00C3E89480E994FF4013E17FC3E8947FE9F5
:10076F0094005002E17F787F7900E17F788079FFF4
:10077F00E820E715C3E52398F84009C3E894014042
:10078F00030207A678010207A6E8F424012523F83F
:10079F0040030207A678FF884B2278A6E6FAA847FF
:1007AF00A948D15AE930E70CC3E89401E994FF4016
:1007BF00160207DAC3E894FFE9940050030207DA40
:1007CF0078FF79000207DA780179FFE920E715C38E
:1007DF00E54B98F84009C3E89401400302080178FB
:1007EF0001020801E8F42401254BF8400302080137
:1007FF0078FF88242278FF20692879A1E76023E514
:10080F0041601F74FF8541F0848539F0306A0375AC
:10081F00F005A4F8C5F0600278FFC3E895645002B4
:10082F00A864886322C3E5409440E5419401E563E1
:10083F005003140145046002F5632202084D22752E
:10084F00E890227883E6FF30EDF9A8BDA9BE0570C8
:10085F00C3E57094084052757000E9FA79A0E7601B
:0F086F0044EA7007E571601B020886C3E89571C3
:10087E006010E5715006600C140208920460F902D3
:10088E000892E571F571C394F6401B7561C0C3946F
:10089E00064013756180C39406400B756140C39486
:1008AE0006400375610075BB0622E561F460020522
:1008BE0061E570B4070375BB1022743279A787F017
:1008CE00A4C5F0A2F733F8C3E895614002A8618889
:1008DE00228824882588268864227540007541F078
:1008EE0022C2AF75C820A8CCA9CDAA3A30CF010A32
:1008FE0075C824D2AFAB3BAC3C883B893CC3E89B6C
:10090E00F8E99C206908F93066024100215AAD3D94
:10091E008A3DF9EA9DFA600678FF79FF213FAE3EE7
:10092E00AF3F8B3E8C3FA83BA93CC3E89EF8E99FA6
:10093E00F9C3E54113FBE54013FAE82AF540E93B1C
:10094E00F54150067540FF7541FF21A7AA40AB4106
:10095E00AC40AD417E047F02C3EB9404400D1E1FDC
:10096E00C3EB94084005206A021E1FC3ED13FDEC75
:10097E0013FCDEF7C3EA9CFAEB9DFBEF6009C3E9BB
:10098E0013F9E813F8DFF7EA28FAEB39FB8A408B04
:10099E004150067BFF8B408B41C3EB94025002D239
:1009AE00663069047F0321D27892E6FFC3E537945F
:1009BE008240110FC3E53794A040010FC3EF940698
:1009CE0040027F057E02E541C4540FF9E541C4544F
:1009DE00F0F8E540C4540F28F8C3E89EFAE99400F5
:1009EE00FB4009C3EA9402EB940050047A02E4FB44
:1009FE00414CAA40AB41EBC4FEEAC4540F4EFCC3BB
:100A0E00EA9CFAEB9400FBC3E813C313F8EA28FA46
:100A1E00EB3400FB8A408B41C3EB94024002C2666A
:100A2E007802EBC4FE7B00EAC4540F4EFAC3EA9878
:100A3E00FA4005C3940250027A027892E6FF3060C3
:100A4E0002414C855192855293D26043E680C3E4B5
:100A5E009AF8E49BF930660241D8E8FAE9FBD3E94B
:100A6E0013FDE813FC88518952C3EF94036038EFED
:100A7E0020E00DE82CF8E93DF9ECFAEDFB020AA1B5
:100A8E00E828F8E939F9C3E82402F8E93400F97ADC
:100A9E00FE7BFFC3EF9403400E8A538B54884D891F
:100AAE004E8C4F8D50610C885389548A4D8B4E8CD1
:100ABE004F8D503069127553F07554FF754FF075A8
:100ACE0050FF7551F07552FF610CE8FAD3E813FC34
:100ADE008851C3EF94036020EF20E007E82CF8EC78
:100AEE00FA41F8E8282402F87AFEC3EF940340088E
:100AFE008A53884D8C4F610C88538A4D8C4FE56814
:100B0E00C3335002646BF5683060026116753402AF
:100B1E00D26043E680E52D54066034A840A941C357
:100B2E00E913F9E813F8C3E913F9E813F830690487
:100B3E00E92440F9C2AF53E67F759100C3E498F5FE
:100B4E0094E499F595759104D26043E680D2AF2274
:100B5E00D264754300752000306C03752040020B83
:100B6E007DD264754300752040306C03752000788B
:100B7E00017901206620E52D54066002C2647914C5
:100B8E00E541C313700104F8C39414400278143085
:100B9E006904781B791B206010E543600C306903F3
:100BAE00D53404D26D8128711E0543E59BF4544063
:100BBE00B52002811230690908C3E8994001186115
:100BCE00A420640A08C3E8994002617D61A4C2644E
:100BDE00C2AF53E67F75910030661275940075951D
:100BEE00F8759104D26043E680D2AF617DE5417E17
:100BFE00FFC3334005C3334001FEC3E49E7594002A
:100C0E00F59561EFC3E53394015002617D306402C6
:100C1E00617DD802812661A4C26DC2AF53E67F7595
:100C2E009100855394855495759104854D92854E0A
:100C3E0093D26043E680D2AFE52D54066008206A59
:100C4E00020533020C64306D0D206C0A206407150A
:100C5E008115810215302278003064027801E53763
:0E0C6E0075F007A4F9E5F028F5F0E9A2F013FF
:100C7C00A2F113A2F213F537C394785003753778A9
:100C8C00C3E53795384008D265C290C291C2923004
:100C9C006002819B854F92855093D26043E68022FF
:100CAC00207D16C2AF754202D294C293306202D23A
:100CBC0092D2AF759F11020E9CC2AF754202D294B4
:100CCC00C295306202D290D2AF759F11020E9C3049
:100CDC007243207D20C2AF754203900139757B10A1
:100CEC00C292D295306204D29181F9C294D2AF757E
:100CFC009F01020E9CC2AF754203900139757B10A7
:100D0C00C290D293306204D291A119C294D2AF7521
:100D1C009F21020E9C207D17C2AF754203900114D7
:100D2C00C292306202D291D2AF759F01020E9CC268
:100D3C00AF754203900114C290306202D291D2AFCF
:100D4C00759F21020E9C207D16C2AF754204D29372
:100D5C00C295306202D291D2AF759F21020E9CC215
:100D6C00AF754204D295C293306202D291D2AF7564
:100D7C009F01020E9C307243207D20C2AF7542054C
:100D8C00900128757B08C291D294306204D290A154
:100D9C009FC293D2AF759F11020E9CC2AF754205D4
:100DAC0090014A757B20C291D294306204D292A1F8
:100DBC00BFC295D2AF759F11020E9C207D17C2AF9A
:100DCC0075420590010AC291306202D290D2AF7581
:100DDC009F11020E9CC2AF75420590011EC291304C
:100DEC0062EBD292D2AF759F11020E9C207D16C27F
:100DFC00AF754206D295C294306202D290D2AF75D2
:100E0C009F01020E9CC2AF754206D293C29430620F
:100E1C0002D292D2AF759F21020E9C307244207D7B
:100E2C0020C2AF75420190014A757B20C290D293CB
:100E3C00306204D292C145C295D2AF759F21020E89
:100E4C009CC2AF754201900128757B08C292D29565
:100E5C00306205D290020E66C293D2AF759F01022A
:100E6C000E9C207D17C2AF75420190011EC29030BE
:100E7C006202D292D2AF759F21020E9CC2AF754214
:100E8C000190010AC292306202D290D2AF759F01DA
:100E9C00C26522900108757B00C290C291C292D2A9
:100EAC0093D294D295C26222788076FF0876FF089E
:100EBC0076FF0876FF08760308760408760B08762A
:100ECC0003087601087601788C76010876FF08769F
:100EDC00FF0876FF0876FF0876FF0876030876FF92
:100EEC000876FF0876FF0876250876D00876FA088B
:100EFC0076FA0876040876FF0876010876000876FC
:100F0C007A0876FF087601087601087600087603E1
:100F1C00087600227887E6FFC272BF0302D272788D
:100F2C0088E6C394036008C27DE630E102D27DC23C
:100F3C007E7889E630E102D27EC3EF9402600875B8
:100F4C008E01D273020F58758E00C273227880E620
:100F5C00149000809378A5F67881E6149000809325
:100F6C0078A6F67886E61490008D9378A7F67886A6
:100F7C00E6F539C394025003753902789CE675384E
:100F8C00FFB402037538A0B4030375388278A3E666
:100F9C001490009A93F566D19F22227896E6FA78FF
:100FAC0097E6FB7888E6B40305C3EB940EFB307F21
:100FBC00047A007BFFC3EB9AFCC3948250027C82C0
:100FCC007572000572EC8572F0A4C3E5F0947D4057
:100FDC00F222D27FF1A71205A11205A17A007B00A3
:100FEC007C10120597E55C2AFA74003BFBDCF37C61
:100FFC0004C3EB13FBEA13FADCF7FEC27F120FA754
:10100C0022757C00757D00E5EF20E6037520000558
:10101C0020903FFFE520146006901DFF14600093A4
:10102C0004600375EF1453D9BF7581C043FF801260
:10103C00059275EF0443B203E5B3240220E70DF5E6
:10104C0021E5E320E0068521B343E301120E9F75F1
:10105C0080FF75A40075F19075D47F75903875A5D7
:0D106C003F75F23F75D50075A60175E24194
:10107900120E9FE4F8F6D8FD756801120EB4121528
:101089008178988673753001C2AF1205AB1205BB22
:101099001205A11205C21205A11205C91205A11254
:1010A90016AA1205AB1205AB1205A6C2AF757C00D4
:1010B900757D0078FA79FA308707D9FBD8F7021CD1
:1010C90000120F20120F59120FA6120FA778988637
:1010D90073120E9F75881075890275C8247591045D
:1010E90075D84075A82275B80275E690759B80750C
:1010F9009D0075D10775BC5875BB0675BA1175E8A1
:1011090080120592D2AF12084A75360053DACF2001
:101119007E0343DA20307E0343DA1043DA01C2D872
:10112900C2711205ABD2617B037A0CE55B70077A59
:101139000CDB030210B41205A12070030210B4C223
:1011490070E55CC3940240E1E52F541F855E5DF5AF
:101159005EB55DD5DAD5C26153DACF207E0343DAB5
:1011690020307E0343DA10C2D8C27178A2E6700833
:10117900D274E52F54E0F52FC2757529001205A622
:10118900307409C3E529940A4002D275120597788B
:10119900023074027800C3E55C9840F0C2AF1205D2
:1011A900BB1205BB1205BBD2AF1205AB754C00785B
:1011B90088E6B4030241B4120597788CE6C394011A
:1011C90050030212B4E530C3940150030212B475FE
:1011D9007CA5757DF1207435C3E55C94FF5003024D
:1011E90012B4C2AF1205D0D2AF1205A6C3E55C9402
:1011F9000150EFC2AF1205BB12059C1205BBD2AF5D
:101209001205A6C3E55C94FF40E902172F7F05D2BA
:101219007F120FA71205A6C2AFC27F120FA7AE5C3D
:10122900C3E55C947FD2AF500241C4120592C2AFAC
:101239001205D0D2AFDFD8120FDEC3EE940578972E
:10124900F61205AB1216B27F0AD27F120FA712054A
:10125900A6C2AFC27F120FA7AE5CC3E55C947FD272
:10126900AF50E4120592C2AF1205BB12059C1205DC
:10127900BBD2AFDFD4120FDEEE24037896F6F879ED
:1012890097E7C394824003985006E824827897F63A
:101299001205AB1215CF1216E11205A6120FA7C33C
:1012A900E55C94FF500221D802172F757C00757DEB
:1012B90000C3E55C954C4003855C4C1205A678019A
:1012C9007988E7B403027805C3E55C98400221B840
:1012D900C2AF1205D01205D01205D0D2AF1205AB9C
:1012E900753000E4F531F5320531E531F4703F052B
:1012F90032789AE67819146012783214600D787D84
:1013090014600878FA146003753200C3E532984016
:101319001D120E9F12059215327531007899867348
:10132900C2AF1205D0D2AF789886731205A61205FE
:101339009CE52A700530740201B4780120740278A2
:1013490006C3E55C9840A17888E6C394036003125C
:1013590005A6E52A70030210B4C2AF120E9FE4F588
:1013690022F523F524F525F526F567D2AF7885E62C
:10137900C333F565E4F544F545F546F547F548F514
:1013890070F52CF52DF53775700875BB101205929F
:1013990012084E30EDFDA8BDA9BEE97001F88871AB
:1013A90012085275700875BB10120F20C2AF756113
:1013B900FF1208C8852261852262852263D2AF7532
:1013C9002201752401752501752601856069756AF3
:1013D900017888E6B40307C27D307602D27DD268EF
:1013E900D269753300120DF8120E271208E8120897
:1013F900EF1208E81208EF1208E8120B6F1206B193
:10140900120C65120CAC1208EF120B5E306E03124F
:1014190006B2206603120804306603120834120C5F
:1014290065120CDB1208EF120B6F306E031206EE19
:10143900120C65120D521208EF120B5E306E031278
:10144900074C120C65120D811208EF120B6F306EEA
:10145900031207A9120C65120DF81208EF12084EB3
:0F146900120B5E120C65120E271208521208EFBA
:1014780030692F856461856462856069756A017960
:10148800187A0CC3E53399400CC269D26A8A35755B
:1014980061FF0214AAC3E55C94014003021403022D
:1014A8001538306A25206C22E535147006C26AD2D8
:1014B8006B8103F535C3E55C94014003021403789E
:1014C80088E6C3940360030215387536007882797C
:1014D800A4E760027803C3E55F985054307404E5CC
:1014E8002A604D7888E6B40317207D05207607A189
:1014F80008307602A108206C07D26C8564618142AD
:1015080078F0306C058564617820C3E54198500215
:101518008103306C1BC26CC27D307602D27DD26AE8
:1015280075351285646181030536E55C6002A13B6F
:10153800753600C2AF120E9F7887E6FE7602120F4C
:10154800207887EEF6E4F522F523F524F525F5262F
:10155800F565752C00752D00D2AF1205A6120E9FE9
:1015680078A4E66006D290D291D292307409C3E58D
:10157800369404400201B441EC901A0D78201216FA
:1015880011E520B45A0CA3121611E520B4A50302E4
:1015980015AF757CA5757DF1120EB41215CF757C4B
:1015A80000757D000215CE901A0378807B0A12160A
:1015B80011A308DBF9901A0F788C7B19121611A366
:1015C80008DBF9901A2822C2AF121654121631906D
:1015D8001A00740E121616A37409121616A374159F
:1015E800121616901A0378807B0A121615A308DBC8
:1015F800F9901A0F788C7B19121615A308DBF912CB
:101608001667121645901A2822E493F622E6438FAD
:1016180001538FFDFFC3E583941C400122EF857CB5
:10162800B7857DB7F0538FFE22438F02438F018524
:101638007CB7857DB7901A0DF0538FFC22901A0D58
:10164800745AD116901A0E74A5D116227A3079D010
:101658007820901A40D111E520F709A3DAF7227A09
:101668003079D0901A40E7D11609A3DAF922AB7481
:10167800A875BB01027984BB02027985BB03027994
:1016880086BB04027992BB05027987BB060279A35F
:10169800BB0702799CBB08027988BB09027989E8F3
:1016A800F7227C051205ABDCFB22C2AF1205BB1288
:1016B80005C21205C91205D012059C1205BB1205F8
:1016C800C21205C91205D012059C1205BB1205C22B
:1016D8001205C91205D0D2AF22C2AF1205D0120529
:1016E800C91205C21205BB12059C1205D01205C904
:1016F8001205C21205BB12059C1205D01205C912AB
:1017080005C21205BBD2AF22AE74AF75C2AF1205C7
:10171800BB1205BB1205BB12059CDEF21205D012E6
:10172800059CDFF8D2AF22D1B2D1AAD1AA75740133
:10173800757501757600F1107C05AD5C1205ABC3BB
:10174800ED955C70F5C3E55C9401400AC3E55C94D3
:10175800FF403202176BD176B1CFD1B2C2AF75EF6D
:1017680014D1AADCD50576C3E5769403500280C669
:10177800D1AA0575E5741490009F93F808C3E57520
:1017880098500280AED1AAD1AA0574C3E574940A10
:101798005002809C120EB4B1CFC2AF75EF14D1AA1B
:0319FD0002100DC8
:101A00000E0915FFFFFFFF03040B0301015AA50197
:101A1000FFFFFFFFFF03FFFFFF25D0FAFA04FF01DE
:091A2000007AFF0101000300FF40
:101A400023585033412320202020202020202020F4
:101A500023424C48454C4923463333302320202031
:101A60002020202020202020202020202020202076
:101C0000C2AFC2D353D9BF7581C043B20343FF8073
:101C1000752438752503B1DC7529A5752AF175E29F
:101C20004043F18053A47F75D4FFD2877DFA7803B7
:101C300079E67C10752200752300901DE97B0675FE
:101C400024987525013087028145208708D8FBD963
:101C5000F9DCF781B7308708D8FBD9F9DCF781B711
:101C6000B19CE493A3C39A6004DDC381B7DBDBB10D
:101C70008E6002812E7B08E493FAA3B16FDBF87AC1
:101C800030B16F752200752300B18EEAFCEBFDC305
:101C9000ED94FE400EB18E8A278B28ED30E0048A49
:101CA000828B83B18E7AC270D8C3ED94FE601950D6
:101CB000CEBD002BEC600F7520007521FF7529004B
:101CC000752A000200008100A827A9280809D80465
:101CD000D90281DCB192EA89AAF281CE0D81A3C337
:101CE000ED94035053EDA2E092007AC5C3E58294CF
:101CF00000E583941C508A200010438F02438F011B
:101D00008529B7852AB7F0300029A827A92808090E
:101D1000438F01538FFDD804D902A133C3E58394C7
:101D20001C4003A3A11689AAE28529B7852AB7F02A
:101D3000A3A116538FFC817F7AC1BD030CE493A34A
:101D4000FAB153DCF8B14B817F8181AA22AB23B178
:101D50006FEBFAEA6222752608C3E52313F523E543
:101D60002213F52250066323A0632201D526EAB18F
:101D7000DCB1DC75260AEAF4200102D287300102C8
:101D8000C287B1DCC3134002C201D526EB22B19257
:101D9000EAFB208702A192308702A197752608AE40
:101DA00024AF25C3EF13FFEE13FEB1E0B1DCC3EAAD
:101DB000133087024480FA30E703632201C3E5232E
:101DC00013F523E52213F52250066323A0632201B5
:101DD000D526D9E52265236523F52222AE24AF2539
:101DE0000E0FDEFEDFFCD20122424C48656C6934E6
:071DF000373164F3300601F6
:00000001FF
